:10000000283084005830A0008001840AA00B042806
:10001000103095002730960000308E0000308F00A1
:10002000013090000B30970007309F008316FF309F
:10003000850083128316CF30860083120C1D1E2884
:100040000C116400A914A9182915A91C2911851BD4
:100050002A282911A91D2D28291127302B0203191F
:100060003828A00020092B05A006A01B3D28442805
:100070000F302A02031C3D284428291D4228AA0FBC
:100080004228AB0A291145282915291D5C2827304B
:100090002D0203195228A00020092D05A006A01B3F
:1000A00057285B280F302C02031C57285B28AC0F05
:1000B0005A28AD0A291160280030AC000030AD008C
:1000C000291D772827302F0203196D28A000200949
:1000D0002F05A006A01B722876280F302E02031CC5
:1000E00072287628AE0F7528AF0A29117B280030B8
:1000F000AE000030AF00291D9228273031020319CD
:100100008828A00020093105A006A01B8D28912871
:100110000F303002031C8D289128B00F9028B10AAF
:10012000291196280030B0000030B100291DAD28FB
:10013000273033020319A328A00020093305A006A5
:10014000A01BA828AC280F303202031CA828AC281A
:10015000B20FAB28B30A2911B1280030B200003029
:10016000B300291DC828273035020319BE28A00076
:1001700020093505A006A01BC328C7280F3034026C
:10018000031CC328C728B40FC628B50A2911CC28D8
:100190000030B4000030B500291DE32827303702B5
:1001A0000319D928A00020093705A006A01BDE28C6
:1001B000E2280F303602031CDE28E228B60FE128C1
:1001C000B70A2911E7280030B6000030B700291D12
:1001D000FE28273039020319F428A0002009390528
:1001E000A006A01BF928FD280F303802031CF928AF
:1001F000FD28B80FFC28B90A291102290030B800DF
:100200000030B900291D192927303B0203190F2995
:10021000A00020093B05A006A01B142918290F30B7
:100220003A02031C14291829BA0F1729BB0A2911ED
:100230001D290030BA000030BB00291D34292730A9
:100240003D0203192A29A00020093D05A006A01B94
:100250002F2933290F303C02031C2F293329BC0FCF
:100260003229BD0A291138290030BC000030BD00F8
:10027000291D4F2927303F0203194529A0002009D5
:100280003F05A006A01B4A294E290F303E02031C41
:100290004A294E29BE0F4D29BF0A29115329003082
:1002A000BE000030BF00291D6A2927304102031912
:1002B0006029A00020094105A006A01B6529692925
:1002C0000F304002031C65296929C00F6829C10A43
:1002D00029116E290030C0000030C10029192916EB
:1002E000291D2912A9182915A91C2911291A7929AA
:1002F0002911291D90292730430203198629A000BE
:1003000020094305A006A01B8B298F290F3042022C
:10031000031C8B298F29C20F8E29C30A2911942906
:100320000030C2000030C300291DAB292730450230
:100330000319A129A00020094505A006A01BA62994
:10034000AA290F304402031CA629AA29C40FA929EF
:10035000C50A2911AF290030C4000030C500291D8D
:10036000C629273047020319BC29A00020094705E8
:10037000A006A01BC129C5290F304602031CC129B4
:10038000C529C60FC429C70A2911CA290030C600C9
:100390000030C700291DE129273049020319D72958
:1003A000A00020094905A006A01BDC29E0290F3088
:1003B0004802031CDC29E029C80FDF29C90A2911DA
:1003C000E5290030C8000030C900291DFC2927306C
:1003D0004B020319F229A00020094B05A006A01B1F
:1003E000F729FB290F304A02031CF729FB29CA0F02
:1003F000FA29CB0A2911002A0030CA000030CB00AC
:10040000291D172A27304D0203190D2AA0002009A3
:100410004D05A006A01B122A162A0F304C02031C01
:10042000122A162ACC0F152ACD0A29111B2A0030B0
:10043000CC000030CD00291D322A27304F0203198D
:10044000282AA00020094F05A006A01B2D2A312A2A
:100450000F304E02031C2D2A312ACE0F302ACF0A2C
:100460002911362A0030CE000030CF00291D4D2A38
:10047000273051020319432AA00020095105A00684
:10048000A01B482A4C2A0F305002031C482A4C2A31
:10049000D00F4B2AD10A2911512A0030D000003048
:1004A000D100291D682A2730530203195E2AA000B3
:1004B00020095305A006A01B632A672A0F305202A9
:1004C000031C632A672AD20F662AD30A29116C2AD1
:1004D0000030D2000030D300291D832A2730550276
:1004E0000319792AA00020095505A006A01B7E2A21
:1004F000822A0F305402031C7E2A822AD40F812ABA
:10050000D50A2911872A0030D4000030D500291DD2
:100510009E2A273057020319942AA0002009570564
:10052000A006A01B992A9D2A0F305602031C992A67
:100530009D2AD60F9C2AD70A2911A22A0030D6005C
:100540000030D700291DB92A273059020319AF2AD4
:10055000A00020095905A006A01BB42AB82A0F3014
:100560005802031CB42AB82AD80FB72AD90A29116D
:10057000BD2A0030D8000030D900291DD42A2730E8
:100580005B020319CA2AA00020095B05A006A01B74
:10059000CF2AD32A0F305A02031CCF2AD32ADA0FCC
:1005A000D22ADB0A2911D82A0030DA000030DB0019
:1005B0002919A916291DA912A9182915A91C29113B
:1005C000A91AE32A2911291DFA2A27305D020319E5
:1005D000F02AA00020095D05A006A01BF52AF92A33
:1005E0000F305C02031CF52AF92ADC0FF82ADD0A19
:1005F0002911FE2A0030DC000030DD00291D152BFA
:1006000027305F0203190B2BA00020095F05A0060D
:10061000A01B102B142B0F305E02031C102B142B6D
:10062000DE0F132BDF0A2911192B0030DE000030FA
:10063000DF00291D302B273061020319262BA00073
:1006400020096105A006A01B2B2B2F2B0F30600269
:10065000031C2B2B2F2BE00F2E2BE10A2911342BFF
:100660000030E0000030E100291D4B2B27306302F1
:100670000319412BA00020096305A006A01B462BEF
:100680004A2B0F306202031C462B4A2BE20F492BE8
:10069000E30A29114F2B0030E2000030E300291D4E
:1006A000662B2730650203195C2BA0002009650525
:1006B000A006A01B612B652B0F306402031C612B6D
:1006C000652BE40F642BE50A29116A2B0030E40046
:1006D0000030E50029192917291D2913A918291502
:1006E000A91C2911291B752B2911291D8C2B0030C0
:1006F00067020319822BA00020096705A006A01B32
:10070000872B8B2B63306602031C872B8B2BE60F0A
:100710008A2BE70A2911902B0030E6000030E70011
:10072000A91B962B0930E8000030E900A917291908
:10073000AE2B003069020319A42BA0002009690523
:10074000A006A01BA92BAD2B09306802031CA92B06
:10075000AD2BE80FAC2BE90A2915B22B0030E800CD
:100760000030E90029196A14291D6A10A9182915F1
:10077000A91C29116A18BD2B2911291DD42B003061
:100780006C020319CA2BA00020096C05A006A01B4F
:10079000CF2BD32B63306B02031CCF2BD32BEB0F50
:1007A000D22BEC0A2911D82B0030EB000030EC00E2
:1007B000291DDE2B0030E6000030E700A9182915BE
:1007C000A91C2911851FE52B29112919EA14291DB6
:1007D000EA106A1DEC2B2911EA186A15EA1C6A1145
:1007E000291DF72BEA19F72BED0FF72BEE0A291924
:1007F000EA15291DEA1100306E020319062CA0002B
:1008000020096E05A006A01B0B2C0D2C01306D02DB
:10081000031C0B2C0D2C29110E2C2915291D252C00
:100820000230700203191B2CA00020097005A006DD
:10083000A01B202C242C57306F02031C202C242CAE
:10084000EF0F232CF00A2911292C0030EF00003083
:10085000F00029196A16291D6A12A9182915A91C60
:100860002911851B342C2911291D3B2CEA1A3B2CFC
:10087000F10F3B2CF20A2919EA16291DEA12003061
:10088000720203194A2CA00020097205A006A01BC1
:100890004F2C512C05307102031C4F2C512C291167
:1008A000522C29156A132919EA17291DEA13EA1F80
:1008B0006E2C003074020319642CA000200974050A
:1008C000A006A01B692C6D2C04307302031C692C3C
:1008D0006D2CF30F6C2CF40AEA13722C0030F30029
:1008E0000030F4007518782C0430F6000030F70062
:1008F0007514EA1B902C003077020319862CA00097
:1009000020097705A006A01B8B2C8F2C04307602C3
:10091000031C8B2C8F2CF60F8E2CF70AEA17942CC5
:100920000030F6000030F700EA1BF514EA1FF5105E
:10093000EA1F9B2C6A172919EA17291DEA13051DBE
:10094000A22CEA13EA1BA915EA1FA911EA1FA92C78
:100950006A176A1B29156A1F2911A9182915A91CCC
:100960002911851BB42C2911291DBA2C0030ED004A
:100970000030EE00A9182915A91C29117511291993
:10098000F515291DF511F518C62CF511F51DC92C05
:1009900075152919F515291DF5116A18D02CF511B1
:1009A000F51DD32C751575192915751D29112919D2
:1009B0000616291D0612A9182915A91C2911061A9F
:1009C000E22C2911291DE82C0030EF000030F00046
:1009D000A9182915A91C2911051BEF2C2911291D5E
:1009E000F52C0030F8000030F900A9182915A91CD1
:1009F000291175122919F516291DF512291A012D2B
:100A0000F512F51E042D75162919F516291DF51276
:100A1000051B0B2DF512F51E0E2D75162919F51651
:100A2000291DF5126A1A152DF512F51E182D7516C9
:100A3000751A2915751E2911291D222D0030F10066
:100A40000030F200A9182915A91C2911851B292D90
:100A500029112919EA14291DEA102919332D751FA6
:100A6000322D2915342D2911EA187517EA1C751332
:100A7000291D3E2D0030AA000030AB00A918291511
:100A8000A91C2911051B452D29112919EA14291D15
:100A9000EA1029194F2DF51F4E2D2915502D29111A
:100AA000EA18F517EA1CF513291D5A2D0030AA0083
:100AB0000030AB00A9182915A91C29117A10291991
:100AC000FA14291DFA10291A662DFA10FA1C692D3C
:100AD0007A142919FA14291DFA10F518702DFA1034
:100AE000FA1C732D7A147A1829157A1C2911291DDC
:100AF0008E2D00302F020319842DA00020092F0510
:100B0000A006A01B892D8D2D09302E02031C892DD6
:100B10008D2DAE0F8C2DAF0A2911922D0030AE0015
:100B20000030AF002919A916291DA912A9182915E5
:100B3000A91C2911A91A9D2D2911291DB42D003098
:100B400031020319AA2DA00020093105A006A01B1F
:100B5000AF2DB32D09303002031CAF2DB32DB00FD4
:100B6000B22DB10A2911B82D0030B0000030B1000B
:100B700029192917291D2913A9182915A91C291173
:100B8000851BC32D291100307C020319CE2DA00036
:100B900020097C05A006A01BD32DDA2D09307B028D
:100BA000031CD32DDA2D291DD82DFB0FD82DFC0ABF
:100BB0002911DB2D291529197A15291D7A11A91852
:100BC0002915A91C29117A19E62D2911A91DE92D2C
:100BD000291129198616291D8612A9182915A91C5B
:100BE0002911291BF42D2911291DFA2D0030FB0094
:100BF0000030FC00A9182915A91C2911851B012EFC
:100C000029112919EA14291DEA1029190B2EFA1D98
:100C10000A2E29150C2E2911EA18FA15EA1CFA11C8
:100C2000291D162E0030FB000030FC008A011E2812
:100C3000FF3FFF3FFF3FFF3FFF3FFF3FFF3FFF3FC4
:100C4000FF3FFF3FFF3FFF3FFF3FFF3FFF3FFF3FB4
:100C5000FF3FFF3FFF3FFF3FFF3FFF3FFF3FFF3FA4
:100C6000FF3FFF3FFF3FFF3FFF3FFF3FFF3FFF3F94
:02400E00503F21
:10420000FF00FF00FF00FF00FF00FF00FF00FF00B6
:10421000FF00FF00FF00FF00FF00FF00FF00FF00A6
:10422000FF00FF00FF00FF00FF00FF00FF00FF0096
:10423000FF00FF00FF00FF00FF00FF00FF00FF0086
:10424000FF00FF00FF00FF00FF00FF00FF00FF0076
:10425000FF00FF00FF00FF00FF00FF00FF00FF0066
:10426000FF00FF00FF00FF00FF00FF00FF00FF0056
:10427000FF00FF00FF00FF00FF00FF00FF00FF0046
:10428000FF00FF00FF00FF00FF00FF00FF00FF0036
:10429000FF00FF00FF00FF00FF00FF00FF00FF0026
:1042A000FF00FF00FF00FF00FF00FF00FF00FF0016
:1042B000FF00FF00FF00FF00FF00FF00FF00FF0006
:1042C000FF00FF00FF00FF00FF00FF00FF00FF00F6
:1042D000FF00FF00FF00FF00FF00FF00FF00FF00E6
:1042E000FF00FF00FF00FF00FF00FF00FF00FF00D6
:1042F000FF00FF00FF00FF00FF00FF00FF00FF00C6
:00000001FF
